:10000000370101007128A948730000008280148123
:10001000988133E6E60009C685050505E389E6FE15
:1000200013351600828052B82A846D242A945D24E8
:10003000E36F85FE52BE8AB8612425C113044006D1
:1000400093045006130940079309300619A08D2C1C
:1000500029C50145592C0808C1450A86C146B52461
:1000600003450101E31585FE03451101E31195FEEA
:1000700003452101E31D25FD03453101E31995FCED
:1000800003454101E31535FD03455101E31125FD0C
:10009000034561014DFD05458ABE0545B9248ABC6D
:1000A000FAB81305C032012413052034ED2A1304D5
:1000B00040369305A0362285FD2A1305E0369305C8
:1000C0003037D52A130A70379305C0375285E52299
:1000D000130BF0379305303C5A85F12A1124930A0B
:1000E0004006930B5006130C4007930C3006930DFB
:1000F000C04093048041130DB04113056038652260
:100100000545E5221305C038792A5D2A21C5014538
:10011000E92A0808C1450A86C146452A0345010166
:10012000E31555FF03451101E31175FF0345210157
:10013000E31D85FD03453101E31975FD03454101CB
:10014000E31595FD03455101E31185FD034561016B
:100150004DFD21A00545512A4DBF1305D039A122DF
:1001600001456122228922859305E03BA9221305DE
:10017000703C152A1305E0369305903D2D2A130592
:10018000C03D1522812A13044500A922E36F85FE94
:1001900052859305603E05221305B03E29221D2A93
:1001A00013044500052AE36F85FE5A859305703FC9
:1001B00019221305D03FC52825223D4409A805452D
:1001C0002D2201451D227D141375F40F3DC993792D
:1001D000F40F6E85C9284E85D9202685E920DD28B3
:1001E00093091500C528E36F35FFD92869D9014562
:1001F000ED280808C1450A86C146C128034501010A
:10020000E31555FF03451101E31175FF0345210176
:10021000E31D85FD03453101E31975FD03454101EA
:10022000E31595FD03455101E31185FD034561018A
:100230004DFD652875206A85BD2061441375F40F56
:1002400059F51305004385205A859305303CA520B8
:100250001305B04389281305E03693053037A128EC
:10026000130580448920BD2013041500A520E36FE9
:1002700085FE52859305C0373D281305304525205E
:10028000912813042500B920E36F85FE4A844A852E
:100290009305A0360D201305D0453120B9BD854802
:1002A0007300000082809148730000008280AD4896
:1002B00073000000828093081008730000008280A1
:1002C0009308500873000000828093087008730040
:1002D00000008280732510C08280732500C0828058
:1002E000930860087300000082800589F322008073
:1002F00093920248B3E2A2007390028082809548F4
:100300007300000082809308000873000000828060
:10031000A148730000008280930830087300000039
:100320008280930840087300000082805553205259
:1003300061696C726F61642043726F7373696E6779
:100340000A00666F72205256436F6E74726F6C6C47
:1003500065720A496E697469616C697A696E6720B1
:1003600048570A006C69676874004F46460062652A
:100370006C6C006F66660067617465007570007371
:1003800069676E616C0049646C650A004C69676856
:10039000747765696768743A204F6E0A0054726119
:1003A000696E2064657465637465640A4C69676886
:1003B000747765696768743A204F66660A00464C30
:1003C000415348524544004C696768743A20466C72
:1003D000617368205265640A006F6E0042656C6C40
:1003E0003A204F6E0A00646F776E00476174653A79
:1003F00020446F776E0A00475245454E00536967A7
:100400006E616C3A20477265656E0A0054696D65CD
:100410006F757420696E2000730A0054696D652041
:10042000726573657420627920747261696E0A0066
:1004300054696D6564206F75740A005369676E6155
:100440006C3A205265640A0042656C6C3A204F6633
:10045000660A00476174653A2055700A004C696766
:0904600068743A204F66660A0038
:00000001FF
